:020000040000FA
:060000000219FD02031CC1
:03000B0002008D63
:03001300020535AE
:03001B0002009050
:03002B000202D1FD
:03005B0002054457
:030073000203097C
:100080000406080C10182030406080A0C0054032E3
:10009000C2AFC2A853E6EFC28E856B8BC0D0D2D35D
:1000A000C0E0C0F0C2CAA8CCA9CDD2CAD2AF758A6E
:1000B00000C3E8956CF8E9956DF9C3E913F9E81305
:1000C000F8E5666007C3E913F9E813F8E97025E875
:1000D000956E4020956E501CE582B410177C007B15
:1000E000007A007908900000A86AE5667004C3E809
:1000F00013F801FD900000D2A8D2AA61E7E0FDC389
:100100009CC39840EF98EB33FB0582E0FCC39DC392
:100110009840E198EB33FB0582E0FDC39CC3984017
:10012000D398EB33FB0582E0FCC39DC39840C59890
:10013000EB33FB0582E0FDC39CC39840B798EB33DB
:10014000FB0582E0FCC39DC39840A998EB33FB05F7
:1001500082E0FDC39CC398409B98EB33FB0582E093
:10016000FCC39DC398408D98EB33FB0582217890AA
:100170000000D2A8D2AA61E7E0FDC39CC39840EF7B
:1001800098EA33FA0582E0FCC39DC39840E198EAFF
:1001900033FA0582E0FDC39CC39840D398EA33FA52
:1001A0000582E0FCC39DC39840C598EA33FA0582F6
:1001B000E0FDC39CC39840B798EA33FA0582E0FC9F
:1001C000C39DC39840A998EA33FA0582E0FDC39C19
:1001D000C398409B98EA33FA0582E0FCC39DC3981C
:1001E000408D98EA33FA0582EBC46B6A54F0F9EA61
:1001F000C454F0C3996009900000D2A8D2AA61E764
:10020000EBF4C454F0F9EAF4C4540F49FAEBF4C423
:10021000540FFBC3EAF99460FAEB9400FB5020C33F
:10022000E97B007A0079006016C3135006F9C39584
:1002300052600AE9F5527553007900800205533087
:100240003A27C3EA94D0F8EB9407F9400BE8FAE9AF
:10025000FB203509D235415D303502C235203902E7
:10026000B235C3EA33FAEB33FBEB2B3B3BF9C3EB81
:1002700013FBEA13FAEA29FAEB3400FB30E3047AC1
:10028000FF7BFFE5255403601B202A18E55D33F949
:10029000EB7007C3E99A4002E9FAE53CC4332AFA55
:1002A000EB3400FBC3EA33C4540FF8EB33C454F00F
:1002B00048F87005EA60027801900000D2A8D2AA3E
:1002C000E5226002152281D4900000D2A8D2AA6152
:1002D000E7C0D0C0E0C2CF0541E5666009E56560D2
:1002E000057565006104756501E52360021523C38A
:1002F000E55460057555006104E5552401F5555038
:10030000037555FFD0E0D0D032C2AF53E67F75926F
:10031000FA7593FFC22053917FD2AF32C0E0E58AD5
:10032000303408856B8BF0A3D0E032D0E0C2AF53FD
:10033000E6EFC0D0C0E0C0F0D2D3D2AF5388EFA870
:100340008AA98CAA40308D010A758A00758C0075C7
:100350004000438810E566700AC3E833F8E933F9D2
:10036000EA33FA30331FE8C4540FFAE9C454F04AB0
:10037000FAC3132AFAC3E833F8E933F9E82AFAE9A9
:100380003406FB61D830320FC3E833E933FAE82A88
:10039000FAE93400FB61D8303115E875F056A4AAAB
:1003A000F0E975F056A42AFAC5F03400FB61D8C311
:1003B000EA13FAE913F9E813F8E875F056A4AAF07D
:1003C000E975F056A42AFAC5F03400C313FBEA130A
:1003D000FAC3EB13FBEA13FAC3EB94125009C3EA16
:1003E0009434EB940750160522E52270021522C3BF
:1003F000E52294325002A128755400A12BE5226019
:100400000215223036067C007D088117AC31AD32F2
:10041000303A04AC33AD34C3EA9CFAEB9DFB92084E
:10042000AE60AF61303A425007203509D235813590
:10043000303502C235303504AE62AF63203902B2C6
:1004400035C3EA33FAEB33FBA208500AEAF424017D
:10045000FAEBF43400FBC3EA9450FAEB9400FB503F
:100460001478007A007B008175A208500878007A21
:10047000007B0081D4E5255403601B202A18E55D2C
:1004800033F9EB7007C3E99A4002E9FAE53CC4335B
:100490002AFAEB3400FBEA8EF0A4F9AAF0EB8EF016
:1004A000A42AFAC5F03400FBC3EB13FDEA13F8C32A
:1004B000ED13FDE813F80FEF146004C3E833F8C33D
:1004C000E933EA33FAEB33FBDFEDEB30E30678FF99
:1004D0007AFF7B078854D230E86003755500C3E586
:1004E0005BFC955C4002AC5CC3EC95545008EC7529
:1004F000F008A4FAABF0EAF4F8EBF45407F9C3E817
:10050000940AFAE99400FB50047A007B008856892B
:10051000578A588B5975230AD0F0D0E0D0D053F7C2
:10052000DF43F74043E6103275230AD0F0D0E0D025
:10053000D043E61032C2AAD28EC2CA85CC6C85CD19
:100540006DD2CA32C2AFC0D0C0E0D2D3A8F9E55A4A
:1005500030E20AE5FA20E23520E132A165E5FA3021
:10056000E22B20E128C3E55713F8E55613F5FB8885
:10057000FCC3E55913F8E55813F5E988EA85575A9D
:1005800053F7BFD2A8303402D2AA53E6EF53F7DFB5
:10059000D0E0D0D0D2AF32790180147903801079C5
:1005A0000A800C791E80087964800479C8800078FC
:1005B00017E4D5E0FDD8FAD9F62278FF202828796B
:1005C000A1E76023E548601F74FF8548F084853FFC
:1005D000F030290375F005A4F8C5F0600278FFC378
:1005E000E8955D5002A85D885C22C3E54794A0E5CC
:1005F000489400E55C500314A1FB046002F55C2202
:1006000075E89022055EC3E55E9408405330EDF432
:10061000A8BDA9BE755E00E9FA79A0E76041EA705D
:1006200006E55F6018800CC3E8955F600EE55F50DB
:1006300005600A1480070460FA8002E55FF55FC375
:100640009569401B755BC0C394044013755B80C300
:100650009404400B755B40C394044003755B002217
:10066000E55B2410500274FFF55B22743279A68793
:10067000F0A4C5F0A2F733F55D227547007548F088
:1006800022C2AFC2CAA8CCA9CDAA4130CF010AD29A
:10069000CAD2AFC3EA13FAE913F9E813F8AB42ACD4
:1006A0004388428943C3E89BF8E99C20280A547F89
:1006B000F9302C02E19FC1F8AD448A44F9EA9D5417
:1006C0007FFA600678FF79FFC1DDAE45AF468B4506
:1006D0008C46A842A943C3E89EF8E99FF9C3E548C0
:1006E00013FBE54713FAE82AF547E93BF5485006BE
:1006F0007547FF7548FFE145AA47AB48AC47AD4891
:100700007E047F02C3EB9404400D1E1FC3EB9408CC
:1007100040052029021E1FC3ED13FDEC13FCDEF77C
:10072000C3EA9CFAEB9DFBEF6009C3E913F9E813F8
:10073000F8DFF7EA28FAEB39FB8A478B4850067B4B
:10074000FF8B478B48C3EB94025002D22C30280415
:100750007F03E1707892E6FFC3E53D948240110F7C
:10076000C3E53D94A040010FC3EF940640027F050E
:100770007E02E548C4540FF9E548C454F0F8E54753
:10078000C4540F28F8C3E89EFAE99400FB4009C35B
:10079000EA9401EB940050047A01E4FB0207EBAA0F
:1007A00047AB48EBC4FEEAC4540F4EFCC3EA9CFAC4
:1007B000EB9400FBC3E813C313F8EA28FAEB340008
:1007C000FB8A478B48C3EB94024002C22C7802EBB1
:1007D000C4FE7B00EAC4540F4EFAC3EA98FA4005FF
:1007E000C3940150027A017892E6FF302002E1EBD7
:1007F000854E92854F93D22043E680C3E49AF8E475
:100800009BF9C3E833F8E933F9302C03020880E898
:10081000FAE9FBD3E913FDE813FC884E894FC3EFD7
:1008200094036038EF20E00CE82CF8E93DF9ECFA8D
:10083000EDFB8013E828F8E939F9C3E82401F8E969
:100840003400F97AFF7BFFC3EF9403400F8A508B8B
:1008500051884A894B8C4C8D4D0208B5885089517E
:100860008A4A8B4B8C4C8D4D3028127550F0755147
:10087000FF754CF0754DFF754EF0754FFF0208B5D2
:10088000E8FAD3E813FC884EC3EF94036021EF200D
:10089000E007E82CF8ECFA01A0E8282401F87AFF38
:1008A000C3EF940340098A50884A8C4C0208B588EB
:1008B000508A4A8C4C30200201B5753A02D220434E
:1008C000E680E5255403602DA847A948C3E913F93C
:1008D000E813F8302804E92440F9C2AF53E67F75E5
:1008E0009100C3E498F594E499F595759104D220AC
:1008F00043E680D2AF22D221754900752000302B0B
:10090000037520402114D221754900752040302BF9
:100910000375200078017901202C20E5255403601F
:1009200002C2217914E548C313700104F8C394147A
:1009300040027814302804781B791BC3E833F8C3CD
:10094000E933F9202010E549600C302803D53A043A
:10095000D22221C711BD0549E59B5440B520022193
:10096000B130280908C3E899400118214320210A21
:1009700008C3E899400221142143C22153E67F7540
:100980009100302C117594007595F0759104D2206A
:1009900043E680020914E5487EFFC3334009C333B0
:1009A0004005C3334001FEC3E49E759400F59521D4
:1009B0008BC3E5399401500221143021022114D84F
:1009C0000221C52143C222C2AF53E67F7591008543
:1009D0005094855195759104854A92854B93D22008
:1009E00043E680D2AFE5255403600720290205398C
:1009F000801030220D202B0A20210715811581023D
:100A000013D22278003021027801E53D75F007A469
:100A1000F9E5F028F5F0E9A2F013A2F113A2F21320
:100A2000F53DC394785003753D78C3E53D953E4050
:100A300009C291C292C29375D57F302002413A8596
:100A40004C92854D93D22043E68022203810C2AFCD
:100A5000C295D29475D537D2AF759F45611BC2AF91
:100A6000C295D29675D56DD2AF759F45611B203862
:100A700010C2AFC29375D55BD294D2AF759F65613A
:100A80001BC2AFC29175D55BD296D2AF759F75610F
:100A90001B203810C2AFC294D29675D55BD2AF7509
:100AA0009F758077C2AFC296D29475D55BD2AF7571
:100AB0009F658067203810C2AFC29275D56DD296FF
:100AC000D2AF759F458054C2AFC29275D537D294CC
:100AD000D2AF759F458044203810C2AFC296D295E0
:100AE00075D56DD2AF759F658031C2AFC294D29576
:100AF00075D537D2AF759F758021203810C2AFC22F
:100B00009175D537D295D2AF759F75800EC2AFC2A1
:100B10009375D56DD295D2AF759F65227A147B7887
:100B200080127A107B8C800C7A0D7BB480067A0B55
:100B30007BC88000E564D5E001227902E4C295D546
:100B4000E0FDD292D5E0FDC292D5E0FDD295D5E090
:100B5000FDE920E002D29130E002D293E564D5E0D5
:100B6000FDE920E002C29130E002C2937496D5E024
:100B7000FDD9C9EAF8D5E0FDD8FBDBB8C29522C2A1
:100B800091C292C293C294C295C29675D57F2278C3
:100B90008076FF0876FF0876FF0876FF0876FF0864
:100BA00076FF0876090876FF087601788C760108CA
:100BB00076FF0876FF0876FF0876FF0876FF08764E
:100BC000030876FF0876FF0876FF0876250876D0BA
:100BD0000876280876500876040876FF087602081A
:100BE00076FF08767A0876FF087607087601087699
:100BF000FF0876FF08760008760022FA75F00CA44C
:100C0000ABF0EAC333F8740133F9E8C333F8E933DE
:100C1000F9E8C32BF8E93400F9E8C333F8E933F90C
:100C2000227888E6C39403D23A5002C23AC238E628
:100C300030E102D238A23892397886E614900080EA
:100C40009378A6F67886E6F53FC394025003753F85
:100C500002789CE6753EFFB40203753EA0B4030320
:100C6000753E8278A0E6F8600674282409D8FCF561
:100C7000697896E671FB88318932789EE671FB8847
:100C80003389347897E671FB88358936717F223055
:100C900036117A007B007CFF7D007E0091F58B6130
:100CA0008A6022303A227896E6FA7B00789EE6FC4B
:100CB0007D00C3EA33FAEB33FBC3EC33FCED33FDC9
:100CC0007E0A91F58B638A627896303A02789EE6C6
:100CD000FA7B007897E6FC7D007E00303A10C3EA8C
:100CE00033FAEB33FBC3EC33FCED33FD7E0A91F5B5
:100CF0008B618A6022C3EC9EFCED9400FDC3EC9AEC
:100D0000FCED9BFDC3EC9423ED940050047C237D0B
:100D100000C3EC94FFED940140047CFF7D017BFF58
:100D20000B7A000AEA7009C3EC33FCED33FDA12015
:100D3000EC8AF0A4AEF0ED8AF0A42E947C40E4EAB4
:100D4000F460DD22D236918F1205A31205A37A003A
:100D50007B007C1012059BE5542AFA74003BFBDCF7
:100D6000F37C04C3EB13FBEA13FADCF7FFEB60023E
:100D70007FFFC236918F2278A5E6F95403D28270A4
:100D800002C282E9540C7000E954307000E954C08A
:100D90007000227567007568007597DE7597AD75F0
:100DA00081C043FF8075EF0675A900717F7580FBD8
:100DB00075F10F75A4047580FB75D4FF75900075EF
:100DC000F27E75A57E75900075D57F75A60175E3D9
:100DD0004075E202717FE4F8F6D8FD718F121416A7
:100DE00078988664753001C2AF1205AB711C12058C
:100DF000A371221205A371281205A3B177C2AF75A2
:100E0000670075680078FA79FA308307D9FBD8F75C
:100E1000021C009121918F78988664717F75A913C7
:100E200075A71075C10075A70075660075E4037598
:100E30008811758E0475890975C80475910475D873
:100E40004075D90875F782759E0375960275DA426A
:100E500075DB4275A82375E69075B801759B8075A2
:100E60009D0075D10C75BCB975BB1075E88075B265
:100E700001120597D2AF753C00C2301205ABC231EA
:100E8000C232C233C234755200755300752200124B
:100E900005A7C3E522940A5002E163D2317522000E
:100EA0001205A7C3E522940A5002E163C231D2328F
:100EB0007522001205A7C3E522940A5002E163756A
:100EC000E4B3758851758E017589AA758C00758D8E
:100ED00000C2A9D2ABD2AA756B80756A14756E5028
:100EE000C232D23475220A1205A7756A10C3E522F0
:100EF000940A7552007553004069758E0C756B002D
:100F0000756A28756E2875220A1205A7756A20C3AE
:100F1000E522940A7552007553004047758E0C7592
:100F20006B80756A14756E1475220A1205A7756AAE
:100F300010C3E522940A755200755300402575E4EC
:100F400003758811758E04758909D2A9C2ABC2AA2E
:100F5000C234D2337522001205A7C3E522940A4099
:100F600002A1FD12059B203003020DFDC2AF711CD2
:100F7000711C711CD2AF1205AB203403303A03024E
:100F8000102212059B788CE6C394015003021022B4
:100F9000E530C3940150030210227567A57568F10E
:100FA0007F02D236918F1205A7C2AFC236918FC38E
:100FB000E554947FD2AF406A120597C2AF712ED22A
:100FC000AFDFDFB144C3EF7897F61205AB1215031C
:100FD0007F0AD236918F1205A7C2AFC236918FC356
:100FE000E554947FD2AF50E8120597C2AF711C123E
:100FF000059F711CD2AFDFDAB144EF24037896F677
:10100000F87997E7C394234003985006E82423789F
:1010100097F61205AB915DB1321205A7120C8F0243
:101020000DFD7567007568001205A7C3E5549401AE
:101030004003020F79C2AF120B2E120B2E120B2E91
:10104000D2AF1205AB753000E4F537F5380537E55A
:1010500037F4703F0538789AE678191460127832C0
:1010600014600D787D14600878FA146003753800F8
:10107000C3E53898401D120B7F1205971538753758
:101080000078998664C2AF120B2ED2AF789886642E
:101090001205A712059FE5237003020DFDC3E55459
:1010A0009401500AC3E5529401501602104D1205E6
:1010B000A7E5237003020DFD75520075530002125F
:1010C00063C3E55294017017C2AF120B7F78998603
:1010D00064120B1C78988664D2AF1205A74155C3E1
:1010E000E55294027017C2AF120B7F789986641292
:1010F0000B2278988664D2AF1205A74155C3E552FA
:1011000094037017C2AF120B7F78998664120B2874
:1011100078988664D2AF1205A74155C3E55294046E
:101120007017C2AF120B7F78998664120B2E7898D5
:101130008664D2AF1205A74155C3E55294057017D6
:10114000C2AF120B7F78998664120B2E7898866452
:10115000D2AF1205A74155C3E55294077019C3E5F4
:101160005394065002019D7401303A02740378884A
:10117000F6C238C2394155C3E55294087019C3E527
:101180005394065002019D7402303A027404788828
:10119000F6D238D2394155C3E55294097017C3E5E8
:1011A0005394065002019D303A0BC37888E69402AE
:1011B000F6C23A4155C3E552940A7016C3E55394FA
:1011C000065002019D203A0A7888E62402F6D23AB7
:1011D0004155C3E55294147025C3E553940650025B
:1011E000019DC2AF901A0B740093D2AF7888F613AA
:1011F000C238C2394002D2384002D2398057C3E5E2
:101200005294157038C3E5539406404FC2AF901AFC
:101210000B740093D2AFF8B801027402B8020274E2
:1012200001B803027404B8040274037888F613C288
:1012300038C2394002D2384002D2398018C3E55250
:10124000940C70117567A57568F1C3E55394064059
:101250000A915DD2AF7552007553007567007568CD
:1012600000019DC2AF120B7FE4D2AFE4F55EF5241E
:10127000F525F53D755E0812059712060030EDFD67
:10128000A8BDA9BEE97001F8885F120604755E0862
:10129000C2AF12066B855D5B855D5CD2AF75A71032
:1012A00075C13075A70075A903756601303A07C28C
:1012B00038303502D238D228753900120AD7120ACE
:1012C000FA12067A12068112067A12068112067A3C
:1012D000120906120A03120A4B1206811208F6209E
:1012E0002C031205BA302C031205EA120A03120A63
:1012F0006E120681120906120A03120A9112068161
:101300001208F6120A03120AB41206811209061212
:101310000A03120AD71206811206001208F6120AF0
:1013200003120AFA120604120681302827855D5B33
:1013300079187A0CC3E53999400EC228D2298A3B24
:10134000855D5B855D5C800CC3E5549401400302C0
:1013500012D061DA30291F202B1CE53B147006C225
:1013600029D22A41D0F53B203A07C3E554940140E5
:10137000030212D08064753C00203A0F78FA79A4F9
:10138000E760027803C3E55598504FE523604B3082
:101390003A17203805203507800F303502800A20A3
:1013A0002B07D22B855D5B610078F0302B05855DC6
:1013B0005B7820C3E5489850030212D0302B1BC243
:1013C0002BC238303502D238D229753B12855D5B8D
:1013D00041D0053CE554600261DD753C00C2AF12AE
:1013E0000B7F75240075250075A91375A71075C1AD
:1013F0000075A700756600D2AF1205A7120B7F78A3
:10140000A4E66006D294D295D296C3E53C940440FB
:1014100003020DFD0148901A0D78209196E520B445
:10142000550AA39196E520B4AA0280137567A575A5
:1014300068F1120B8F915D756700756800801D90D3
:101440001A0378807B0A9196A308DBFA901A0F782A
:101450008C7B1A9196A308DBFA901A2922C2AF91CD
:10146000D991B6901A007410919BA37407919BA315
:101470007421919B901A0378807B0A919AA308DBD0
:10148000FA901A0F788C7B1A919AA308DBFA91ECE8
:1014900091CA901A2922E493F622E6438F01538FD2
:1014A000FDFFC3E583941C400122EF8567B7856883
:1014B000B7F0538FFE22438F02438F018567B785B4
:1014C00068B7901A0DF0538FFC22901A0D74559145
:1014D0009B901A0E74AA919B227A3079D078209032
:1014E0001A409196E520F709A3DAF7227A3079D0ED
:1014F000901A40E7919B09A3DAF9227C051205AB0B
:10150000DCFB22C2AF120B1C120B22120B28120B97
:101510002E12059F120B1C120B22120B28120B2EDF
:1015200012059F120B1C120B22120B28120B2ED22B
:10153000AF22C2AF120B2E120B28120B22120B1C61
:1015400012059F120B2E120B28120B22120B1C12CB
:10155000059F120B2E120B28120B22120B1CD2AF5E
:011560002268
:1019FD00020D93100721FFFFFFFFFFFF09FF01FFFE
:101A0D0055AA01FFFFFFFFFF03FFFFFF25D0285061
:0D1A1D0004FF02FF7AFF0701FFFF0000FF3A
:101A4000234D5F485F303523202020202020202098
:101A500023424C48454C492445464D3842323123B7
:101A60002020202020202020202020202020202076
:101C0000C2AFC2D37597DE7597AD7581C075A90057
:101C100043FF80752438752503B1DB7529A5752A26
:101C2000F143F10853A4F7D28375D4FF75E3407DE7
:101C3000FA780379E67C10752200752300901DE880
:101C40007B0675249875250130830281482083081E
:101C5000D8FBD9F9DCF781BA308308D8FBD9F9DC95
:101C6000F781BAB19BE493A3C39A6004DDC381BA40
:101C7000DBDBB18D600281317B08E493FAA3B16EA6
:101C8000DBF87A30B16E752200752300B18DEAFC65
:101C9000EBFDC3ED94FE400EB18D8A278B28ED300D
:101CA000E0048A828B83B18D7AC270D8C3ED94FE32
:101CB000601950CEBD0029EC600F7520007521FF22
:101CC000752900752A000200008100A827A92808AC
:101CD00009D804D90281DDB191EAF281D10D81A642
:101CE000C3ED94035051EDA2E092007AC5C3E582A2
:101CF0009400E583941C508C200010438F02438F86
:101D0000018529B7852AB7F0300027A827A9280818
:101D100009438F01538FFDD804D902A132C3E58353
:101D2000941C4003A3A117E28529B7852AB7F0A325
:101D3000A117538FFC81827AC1BD030CE493A3FAEF
:101D4000B152DCF8B14A81828184AA22AB23B16E00
:101D5000EBFAEA6222752608C3E52313F523E52290
:101D600013F52250066323A0632201D526EAB1DBD6
:101D7000B1DB75260AEAF4200102D283300102C2E7
:101D800083B1DBC3134002C201D526EB22B191EA35
:101D9000FB208302A191308302A196752608AE2410
:101DA000AF25C3EF13FFEE13FEB1DFB1DBC3EA13C0
:101DB0003083024480FA30E703632201C3E5231332
:101DC000F523E52213F52250066323A0632201D5F3
:101DD00026D9E52265236523F52222AE24AF250E00
:101DE0000FDEFEDFFCD20122424C48656C693437BD
:061DF0003164E8B20601B7
:00000001FF
